
 COMPOBJ

 Start     Length     Name                   Class
 0001:0000 04340H     SEG_CODE_TEXT          CODE
 0001:4340 00C08H     _TEXT                  CODE
 0001:4F50 00184H     COMDAT_SEG1            CODE
 0002:0000 00048H     SEG_CODE5_DATA         FAR_DATA
 0003:0000 00010H     NULL                   BEGDATA
 0003:0010 0029EH     _DATA                  DATA
 0003:02AE 00000H     XIFCB                  DATA
 0003:02AE 00004H     XIFU                   DATA
 0003:02B2 00000H     XIFL                   DATA
 0003:02B2 00000H     XIFM                   DATA
 0003:02B2 00000H     XIFCE                  DATA
 0003:02B2 0000EH     CDATA                  DATA
 0003:02C0 00000H     XIFB                   DATA
 0003:02C0 00000H     XIF                    DATA
 0003:02C0 00000H     XIFE                   DATA
 0003:02C0 00000H     XIB                    DATA
 0003:02C0 00000H     XI                     DATA
 0003:02C0 00000H     XIE                    DATA
 0003:02C0 00000H     XPB                    DATA
 0003:02C0 00000H     XP                     DATA
 0003:02C0 00000H     XPE                    DATA
 0003:02C0 00000H     XCB                    DATA
 0003:02C0 00000H     XC                     DATA
 0003:02C0 00000H     XCE                    DATA
 0003:02C0 00000H     XCFB                   DATA
 0003:02C0 00000H     XCFCRT                 DATA
 0003:02C0 00000H     XCF                    DATA
 0003:02C0 00000H     XCFE                   DATA
 0003:02C0 00000H     DBDATA                 DATA
 0003:02C0 00000H     CONST                  CONST
 0003:02C0 00008H     HDR                    MSG
 0003:02C8 0016EH     MSG                    MSG
 0003:0436 00002H     PAD                    MSG
 0003:0438 00001H     EPAD                   MSG
 0003:043A 00092H     _BSS                   BSS
 0003:04CC 00000H     XOB                    BSS
 0003:04CC 00084H     XO                     BSS
 0003:0550 00000H     XOE                    BSS
 0003:0550 00000H     XOFB                   BSS
 0003:0550 00000H     XOF                    BSS
 0003:0550 00000H     XOFE                   BSS

 Origin   Group
 0003:0   DGROUP

 Address   Export                  Alias

 0001:31FC ??0CArrayFValue@@REC@KI@Z  ??0CArrayFValue@@REC@KI@Z
 0001:377E ??0CMapKeyToValue@@REC@KIIHP7CIPEXI@ZI@Z  ??0CMapKeyToValue@@REC@KIIHP7CIPEXI@ZI@Z
 0001:325A ??1CArrayFValue@@REC@XZ  ??1CArrayFValue@@REC@XZ
 0001:3822 ??1CMapKeyToValue@@REC@XZ  ??1CMapKeyToValue@@REC@XZ
 0001:4FFA ?AddRef@CStdMalloc@@VEAKXZ  ?AddRef@CStdMalloc@@VEAKXZ
 0001:2610 ?Alloc@CStdMalloc@@VEAPEXK@Z  ?Alloc@CStdMalloc@@VEAPEXK@Z
 0001:3770 ?AssertValid@CArrayFValue@@RFCXXZ  ?AssertValid@CArrayFValue@@RFCXXZ
 0001:4282 ?AssertValid@CMapKeyToValue@@RFCXXZ  ?AssertValid@CMapKeyToValue@@RFCXXZ
 0001:3BBC ?CompareAssocKey@CMapKeyToValue@@BFCHPEUCAssoc@1@PEXI@Z  ?CompareAssocKey@CMapKeyToValue@@BFCHPEUCAssoc@1@PEXI@Z
 0001:2864 ?DidAlloc@CStdMalloc@@VEAHPEX@Z  ?DidAlloc@CStdMalloc@@VEAHPEX@Z
 0001:27AE ?Free@CStdMalloc@@VEAXPEX@Z  ?Free@CStdMalloc@@VEAXPEX@Z
 0001:3ADE ?FreeAssoc@CMapKeyToValue@@BECXPEUCAssoc@1@@Z  ?FreeAssoc@CMapKeyToValue@@BECXPEUCAssoc@1@@Z
 0001:3CEA ?FreeAssocKey@CMapKeyToValue@@BFCXPEUCAssoc@1@@Z  ?FreeAssocKey@CMapKeyToValue@@BFCXPEUCAssoc@1@@Z
 0001:3444 ?FreeExtra@CArrayFValue@@RECXXZ  ?FreeExtra@CArrayFValue@@RECXXZ
 0001:3B1E ?GetAssocAt@CMapKeyToValue@@BFCPEUCAssoc@1@PEXIAEI@Z  ?GetAssocAt@CMapKeyToValue@@BFCPEUCAssoc@1@PEXIAEI@Z
 0001:3C94 ?GetAssocKeyPtr@CMapKeyToValue@@BFCXPEUCAssoc@1@PEPEXPEI@Z  ?GetAssocKeyPtr@CMapKeyToValue@@BFCXPEUCAssoc@1@PEPEXPEI@Z
 0001:3D46 ?GetAssocValue@CMapKeyToValue@@BFCXPEUCAssoc@1@PEX@Z  ?GetAssocValue@CMapKeyToValue@@BFCXPEUCAssoc@1@PEX@Z
 0001:3D1E ?GetAssocValuePtr@CMapKeyToValue@@BFCXPEUCAssoc@1@PEPEX@Z  ?GetAssocValuePtr@CMapKeyToValue@@BFCXPEUCAssoc@1@PEPEX@Z
 0000:0000 ?GetCount@CMapKeyToValue@@RFCHXZ  ?GetCount@CMapKeyToValue@@RFCHXZ
 0001:4114 ?GetHKey@CMapKeyToValue@@RFCKPEXI@Z  ?GetHKey@CMapKeyToValue@@RFCKPEXI@Z
 0001:415C ?GetNextAssoc@CMapKeyToValue@@RFCXPEPEXPEXPEI1@Z  ?GetNextAssoc@CMapKeyToValue@@RFCXPEPEXPEXPEI1@Z
 0001:3280 ?GetSize@CArrayFValue@@RFCHXZ  ?GetSize@CArrayFValue@@RFCHXZ
 0001:27F8 ?GetSize@CStdMalloc@@VEAKPEX@Z  ?GetSize@CStdMalloc@@VEAKPEX@Z
 0001:413C ?GetStartPosition@CMapKeyToValue@@RFCPEXXZ  ?GetStartPosition@CMapKeyToValue@@RFCPEXXZ
 0001:28AA ?HeapMinimize@CStdMalloc@@VEAXXZ  ?HeapMinimize@CStdMalloc@@VEAXXZ
 0001:36A2 ?IndexOf@CArrayFValue@@RECHPEXII@Z  ?IndexOf@CArrayFValue@@RECHPEXII@Z
 0001:387E ?InitHashTable@CMapKeyToValue@@BECHXZ  ?InitHashTable@CMapKeyToValue@@BECHXZ
 0001:3568 ?InsertAt@CArrayFValue@@RECHHPEXH@Z  ?InsertAt@CArrayFValue@@RECHHPEXH@Z
 0001:3DE2 ?Lookup@CMapKeyToValue@@RFCHPEXI0@Z  ?Lookup@CMapKeyToValue@@RFCHPEXI0@Z
 0001:3E6E ?LookupAdd@CMapKeyToValue@@RFCHPEXI0@Z  ?LookupAdd@CMapKeyToValue@@RFCHPEXI0@Z
 0001:3E1C ?LookupHKey@CMapKeyToValue@@RFCHKPEX@Z  ?LookupHKey@CMapKeyToValue@@RFCHKPEX@Z
 0001:39B2 ?NewAssoc@CMapKeyToValue@@BECPEUCAssoc@1@IPEXI0@Z  ?NewAssoc@CMapKeyToValue@@BECPEUCAssoc@1@IPEXI0@Z
 0001:216C ?Proxy1632AddRef@@ZAKPEVCProxy1632@@@Z  ?Proxy1632AddRef@@ZAKPEVCProxy1632@@@Z
 0001:2282 ?Proxy1632Method10@@ZAKPEVCProxy1632@@@Z  ?Proxy1632Method10@@ZAKPEVCProxy1632@@@Z
 0001:229C ?Proxy1632Method11@@ZAKPEVCProxy1632@@@Z  ?Proxy1632Method11@@ZAKPEVCProxy1632@@@Z
 0001:22B6 ?Proxy1632Method12@@ZAKPEVCProxy1632@@@Z  ?Proxy1632Method12@@ZAKPEVCProxy1632@@@Z
 0001:22D0 ?Proxy1632Method13@@ZAKPEVCProxy1632@@@Z  ?Proxy1632Method13@@ZAKPEVCProxy1632@@@Z
 0001:22EA ?Proxy1632Method14@@ZAKPEVCProxy1632@@@Z  ?Proxy1632Method14@@ZAKPEVCProxy1632@@@Z
 0001:2304 ?Proxy1632Method15@@ZAKPEVCProxy1632@@@Z  ?Proxy1632Method15@@ZAKPEVCProxy1632@@@Z
 0001:231E ?Proxy1632Method16@@ZAKPEVCProxy1632@@@Z  ?Proxy1632Method16@@ZAKPEVCProxy1632@@@Z
 0001:2338 ?Proxy1632Method17@@ZAKPEVCProxy1632@@@Z  ?Proxy1632Method17@@ZAKPEVCProxy1632@@@Z
 0001:2352 ?Proxy1632Method18@@ZAKPEVCProxy1632@@@Z  ?Proxy1632Method18@@ZAKPEVCProxy1632@@@Z
 0001:236C ?Proxy1632Method19@@ZAKPEVCProxy1632@@@Z  ?Proxy1632Method19@@ZAKPEVCProxy1632@@@Z
 0001:2386 ?Proxy1632Method20@@ZAKPEVCProxy1632@@@Z  ?Proxy1632Method20@@ZAKPEVCProxy1632@@@Z
 0001:23A0 ?Proxy1632Method21@@ZAKPEVCProxy1632@@@Z  ?Proxy1632Method21@@ZAKPEVCProxy1632@@@Z
 0001:23BA ?Proxy1632Method22@@ZAKPEVCProxy1632@@@Z  ?Proxy1632Method22@@ZAKPEVCProxy1632@@@Z
 0001:23D4 ?Proxy1632Method23@@ZAKPEVCProxy1632@@@Z  ?Proxy1632Method23@@ZAKPEVCProxy1632@@@Z
 0001:23EE ?Proxy1632Method24@@ZAKPEVCProxy1632@@@Z  ?Proxy1632Method24@@ZAKPEVCProxy1632@@@Z
 0001:2408 ?Proxy1632Method25@@ZAKPEVCProxy1632@@@Z  ?Proxy1632Method25@@ZAKPEVCProxy1632@@@Z
 0001:2422 ?Proxy1632Method26@@ZAKPEVCProxy1632@@@Z  ?Proxy1632Method26@@ZAKPEVCProxy1632@@@Z
 0001:243C ?Proxy1632Method27@@ZAKPEVCProxy1632@@@Z  ?Proxy1632Method27@@ZAKPEVCProxy1632@@@Z
 0001:2456 ?Proxy1632Method28@@ZAKPEVCProxy1632@@@Z  ?Proxy1632Method28@@ZAKPEVCProxy1632@@@Z
 0001:2470 ?Proxy1632Method29@@ZAKPEVCProxy1632@@@Z  ?Proxy1632Method29@@ZAKPEVCProxy1632@@@Z
 0001:248A ?Proxy1632Method30@@ZAKPEVCProxy1632@@@Z  ?Proxy1632Method30@@ZAKPEVCProxy1632@@@Z
 0001:24A4 ?Proxy1632Method31@@ZAKPEVCProxy1632@@@Z  ?Proxy1632Method31@@ZAKPEVCProxy1632@@@Z
 0001:21CC ?Proxy1632Method3@@ZAKPEVCProxy1632@@@Z  ?Proxy1632Method3@@ZAKPEVCProxy1632@@@Z
 0001:21E6 ?Proxy1632Method4@@ZAKPEVCProxy1632@@@Z  ?Proxy1632Method4@@ZAKPEVCProxy1632@@@Z
 0001:2200 ?Proxy1632Method5@@ZAKPEVCProxy1632@@@Z  ?Proxy1632Method5@@ZAKPEVCProxy1632@@@Z
 0001:221A ?Proxy1632Method6@@ZAKPEVCProxy1632@@@Z  ?Proxy1632Method6@@ZAKPEVCProxy1632@@@Z
 0001:2234 ?Proxy1632Method7@@ZAKPEVCProxy1632@@@Z  ?Proxy1632Method7@@ZAKPEVCProxy1632@@@Z
 0001:224E ?Proxy1632Method8@@ZAKPEVCProxy1632@@@Z  ?Proxy1632Method8@@ZAKPEVCProxy1632@@@Z
 0001:2268 ?Proxy1632Method9@@ZAKPEVCProxy1632@@@Z  ?Proxy1632Method9@@ZAKPEVCProxy1632@@@Z
 0001:20FE ?Proxy1632QueryInterface@@ZAKPEVCProxy1632@@AFUGUID@@PEPEX@Z  ?Proxy1632QueryInterface@@ZAKPEVCProxy1632@@AFUGUID@@PEPEX@Z
 0001:219C ?Proxy1632Release@@ZAKPEVCProxy1632@@@Z  ?Proxy1632Release@@ZAKPEVCProxy1632@@@Z
 0001:4F50 ?QueryInterface@CStdMalloc@@VEAPEXAFUGUID@@PEPEX@Z  ?QueryInterface@CStdMalloc@@VEAPEXAFUGUID@@PEPEX@Z
 0001:268E ?Realloc@CStdMalloc@@VEAPEXPEXK@Z  ?Realloc@CStdMalloc@@VEAPEXPEXK@Z
 0001:501C ?Release@CStdMalloc@@VEAKXZ  ?Release@CStdMalloc@@VEAKXZ
 0001:38F0 ?RemoveAll@CMapKeyToValue@@RECXXZ  ?RemoveAll@CMapKeyToValue@@RECXXZ
 0001:364A ?RemoveAt@CArrayFValue@@RECXHH@Z  ?RemoveAt@CArrayFValue@@RECXHH@Z
 0001:406C ?RemoveHKey@CMapKeyToValue@@RECHK@Z  ?RemoveHKey@CMapKeyToValue@@RECHK@Z
 0001:3FAE ?RemoveKey@CMapKeyToValue@@RECHPEXI@Z  ?RemoveKey@CMapKeyToValue@@RECHPEXI@Z
 0001:3C10 ?SetAssocKey@CMapKeyToValue@@BFCHPEUCAssoc@1@PEXI@Z  ?SetAssocKey@CMapKeyToValue@@BFCHPEUCAssoc@1@PEXI@Z
 0001:3D84 ?SetAssocValue@CMapKeyToValue@@BFCXPEUCAssoc@1@PEX@Z  ?SetAssocValue@CMapKeyToValue@@BFCXPEUCAssoc@1@PEX@Z
 0001:34F6 ?SetAt@CArrayFValue@@RECXHPEX@Z  ?SetAt@CArrayFValue@@RECXHPEX@Z
 0001:3EB6 ?SetAt@CMapKeyToValue@@RECHPEXI0@Z  ?SetAt@CMapKeyToValue@@RECHPEXI0@Z
 0001:352A ?SetAtGrow@CArrayFValue@@RECHHPEX@Z  ?SetAtGrow@CArrayFValue@@RECHHPEX@Z
 0001:3F72 ?SetAtHKey@CMapKeyToValue@@RECHKPEX@Z  ?SetAtHKey@CMapKeyToValue@@RECHKPEX@Z
 0001:3296 ?SetSize@CArrayFValue@@RECHHH@Z  ?SetSize@CArrayFValue@@RECHHH@Z
 0000:0000 ?SizeAssoc@CMapKeyToValue@@BFCIXZ  ?SizeAssoc@CMapKeyToValue@@BFCIXZ
 0001:1C70 ?Sm16RhAddRef@@ZAKPEVCSm16ReleaseHandler@@@Z  ?Sm16RhAddRef@@ZAKPEVCSm16ReleaseHandler@@@Z
 0001:1C92 ?Sm16RhQI@@ZAPEXPEVCSm16ReleaseHandler@@AFUGUID@@PEPEX@Z  ?Sm16RhQI@@ZAPEXPEVCSm16ReleaseHandler@@AFUGUID@@PEPEX@Z
 0001:1CE4 ?Sm16RhRelease@@ZAKPEVCSm16ReleaseHandler@@@Z  ?Sm16RhRelease@@ZAKPEVCSm16ReleaseHandler@@@Z
 0001:34D6 ?_GetAt@CArrayFValue@@RFCPEXH@Z  ?_GetAt@CArrayFValue@@RFCPEXH@Z
 0001:1F1C ADDAPPCOMPATFLAG        ADDAPPCOMPATFLAG
 0001:162A CALL32INITIALIZE        CALL32INITIALIZE
 0001:1814 CALL32UNINITIALIZE      CALL32UNINITIALIZE
 0001:18BC CALLOBJECTINWOW         CALLOBJECTINWOW
 0001:1954 CALLOBJECTINWOWCHECKINIT  CALLOBJECTINWOWCHECKINIT
 0001:19BC CALLOBJECTINWOWCHECKTHKMGR  CALLOBJECTINWOWCHECKTHKMGR
 0001:188E CALLTHKMGRINITIALIZE    CALLTHKMGRINITIALIZE
 0001:1860 CALLTHKMGRUNINITIALIZE  CALLTHKMGRUNINITIALIZE
 0001:1264 CLSIDFROMOLE1CLASS      CLSIDFROMOLE1CLASS
 0001:023C CLSIDFROMPROGID         CLSIDFROMPROGID
 0001:0000 CLSIDFROMSTRING         CLSIDFROMSTRING
 0001:0AB0 COBUILDVERSION          COBUILDVERSION
 0001:0262 COCREATEGUID            COCREATEGUID
 0001:01CA COCREATEINSTANCE        COCREATEINSTANCE
 0001:2946 COCREATESTANDARDMALLOC  COCREATESTANDARDMALLOC
 0001:0132 CODISCONNECTOBJECT      CODISCONNECTOBJECT
 0001:02AE CODOSDATETIMETOFILETIME  CODOSDATETIMETOFILETIME
 0001:02D4 COFILETIMENOW           COFILETIMENOW
 0001:0288 COFILETIMETODOSDATETIME  COFILETIMETODOSDATETIME
 0001:3186 COFREEALLLIBRARIES      COFREEALLLIBRARIES
 0001:315A COFREELIBRARY           COFREELIBRARY
 0001:31BC COFREEUNUSEDLIBRARIES   COFREEUNUSEDLIBRARIES
 0001:122E COGETCLASSEXT           COGETCLASSEXT
 0001:004E COGETCLASSOBJECT        COGETCLASSOBJECT
 0001:0A86 COGETCURRENTPROCESS     COGETCURRENTPROCESS
 0001:081E COGETMALLOC             COGETMALLOC
 0001:017E COGETSTANDARDMARSHAL    COGETSTANDARDMARSHAL
 0001:093C COGETSTATE              COGETSTATE
 0001:0320 COGETTREATASCLASS       COGETTREATASCLASS
 0001:12BE COHANDLEINCOMINGCALL    COHANDLEINCOMINGCALL
 0001:056E COINITIALIZE            COINITIALIZE
 0001:01A4 COISHANDLERCONNECTED    COISHANDLERCONNECTED
 0001:01F0 COISOLE1CLASS           COISOLE1CLASS
 0001:3128 COLOADLIBRARY           COLOADLIBRARY
 0001:0158 COLOCKOBJECTEXTERNAL    COLOCKOBJECTEXTERNAL
 0001:0AC2 COMARSHALHRESULT        COMARSHALHRESULT
 0001:00C0 COMARSHALINTERFACE      COMARSHALINTERFACE
 0001:2A74 COMEMALLOC              COMEMALLOC
 0001:29F2 COMEMCTXOF              COMEMCTXOF
 0001:2AEC COMEMFREE               COMEMFREE
 0001:1EB8 CONVERTHR1632           CONVERTHR1632
 0001:1EEA CONVERTHR3216           CONVERTHR3216
 0001:1276 COOPENCLASSKEY          COOPENCLASSKEY
 0001:0074 COREGISTERCLASSOBJECT   COREGISTERCLASSOBJECT
 0001:02FA COREGISTERMESSAGEFILTER  COREGISTERMESSAGEFILTER
 0001:010C CORELEASEMARSHALDATA    CORELEASEMARSHALDATA
 0001:009A COREVOKECLASSOBJECT     COREVOKECLASSOBJECT
 0001:12AC CORUNMODALLOOP          CORUNMODALLOOP
 0001:121C COSETACKSTATE           COSETACKSTATE
 0001:09D6 COSETSTATE              COSETSTATE
 0001:0346 COTREATASCLASS          COTREATASCLASS
 0001:0796 COUNINITIALIZE          COUNINITIALIZE
 0001:0B44 COUNMARSHALHRESULT      COUNMARSHALHRESULT
 0001:00E6 COUNMARSHALINTERFACE    COUNMARSHALINTERFACE
 0001:119E FNASSERT                FNASSERT
 0001:1148 GETSCODE                GETSCODE
 0001:0D3C GUIDFROMSTRING          GUIDFROMSTRING
 0001:1050 IIDFROMSTRING           IIDFROMSTRING
 0001:0BE8 ISEQUALGUID             ISEQUALGUID
 0001:2C90 ISVALIDIID              ISVALIDIID
 0001:2C22 ISVALIDINTERFACE        ISVALIDINTERFACE
 0001:2BDA ISVALIDPTRIN            ISVALIDPTRIN
 0001:2BFE ISVALIDPTROUT           ISVALIDPTROUT
 0001:1344 LOOKUPETASK             LOOKUPETASK
 0001:1240 LRPCCALL                LRPCCALL
 0001:11B0 LRPCDISPATCH            LRPCDISPATCH
 0001:11F8 LRPCFREEMONITORDATA     LRPCFREEMONITORDATA
 0001:1288 LRPCGETTHREADWINDOW     LRPCGETTHREADWINDOW
 0001:1252 LRPCREGISTERMONITOR     LRPCREGISTERMONITOR
 0001:129A LRPCREVOKEMONITOR       LRPCREVOKEMONITOR
 0001:383A MKVDEFAULTHASHKEY       MKVDEFAULTHASHKEY
 0001:12E2 OLE1CLASSFROMCLSID2     OLE1CLASSFROMCLSID2
 0001:0216 PROGIDFROMCLSID         PROGIDFROMCLSID
 0001:1178 PROPAGATERESULT         PROPAGATERESULT
 0001:11E6 REMALLOCOID             REMALLOCOID
 0001:11C2 REMCONNECTTOOBJECT      REMCONNECTTOOBJECT
 0001:11D4 REMCREATEREMOTEHANDLER  REMCREATEREMOTEHANDLER
 0001:1306 REMFREEOID              REMFREEOID
 0001:12D0 REMGETINFOFORCID        REMGETINFOFORCID
 0001:12F4 REMLOOKUPSHUNK          REMLOOKUPSHUNK
 0001:157A REMOVEETASK             REMOVEETASK
 0001:1160 RESULTFROMSCODE         RESULTFROMSCODE
 0001:13FE SETETASK                SETETASK
 0001:1908 SSCALLOBJECTINWOW       SSCALLOBJECTINWOW
 0001:0EEC STRINGFROMCLSID         STRINGFROMCLSID
 0001:10DE STRINGFROMGUID2         STRINGFROMGUID2
 0001:0FA2 STRINGFROMIID           STRINGFROMIID
 0001:120A TIMERCALLBACKPROC       TIMERCALLBACKPROC
 0001:039E WEP                     WEP
 0001:1FAE _CLSID_StdMarshal       _CLSID_StdMarshal
 0001:1F7E _GUID_NULL              _GUID_NULL
 0001:203E _IID_IBindCtx           _IID_IBindCtx
 0001:1F5E _IID_IClassFactory      _IID_IClassFactory
 0001:1FEE _IID_IDfReserved1       _IID_IDfReserved1
 0001:1FDE _IID_IDfReserved2       _IID_IDfReserved2
 0001:1FCE _IID_IDfReserved3       _IID_IDfReserved3
 0001:204E _IID_IEnumSTATSTG       _IID_IEnumSTATSTG
 0001:1F8E _IID_IExternalConnection  _IID_IExternalConnection
 0001:200E _IID_IInternalMoniker   _IID_IInternalMoniker
 0001:207E _IID_ILockBytes         _IID_ILockBytes
 0001:1F4E _IID_IMalloc            _IID_IMalloc
 0001:20EE _IID_IMarshal           _IID_IMarshal
 0001:1FBE _IID_IMessageFilter     _IID_IMessageFilter
 0001:202E _IID_IMoniker           _IID_IMoniker
 0001:209E _IID_IProxyManager      _IID_IProxyManager
 0001:208E _IID_IPSFactory         _IID_IPSFactory
 0001:1FFE _IID_IRootStorage       _IID_IRootStorage
 0001:20DE _IID_IRpcChannel        _IID_IRpcChannel
 0001:20AE _IID_IRpcProxy          _IID_IRpcProxy
 0001:20CE _IID_IRpcStub           _IID_IRpcStub
 0001:201E _IID_IRunningObjectTable  _IID_IRunningObjectTable
 0001:1F9E _IID_IStdMarshalInfo    _IID_IStdMarshalInfo
 0001:206E _IID_IStorage           _IID_IStorage
 0001:205E _IID_IStream            _IID_IStream
 0001:20BE _IID_IStubManager       _IID_IStubManager
 0001:1F6E _IID_IUnknown           _IID_IUnknown
 0001:4ECA ___ExportedStub         ___ExportedStub

  Address         Publics by Name

 0001:31FC       ??0CArrayFValue@@REC@KI@Z
 0001:377E       ??0CMapKeyToValue@@REC@KIIHP7CIPEXI@ZI@Z
 0001:5058       ??0IMalloc@@REC@XZ
 0001:325A       ??1CArrayFValue@@REC@XZ
 0001:3822       ??1CMapKeyToValue@@REC@XZ
 0001:442A       ??2@ZAPEXI@Z
 0001:4418       ??3@ZAXPEX@Z
 0001:50B0       ??_7CStdMalloc@@6F@
 0001:508C       ??_7IMalloc@@6F@
 0001:5080       ??_7IUnknown@@6F@
 0001:1BF4       ?AddRef16@@ZCKPEUIUnknown@@@Z
 0001:4FFA       ?AddRef@CStdMalloc@@VEAKXZ
 0001:2610       ?Alloc@CStdMalloc@@VEAPEXK@Z
 0001:24BE       ?AllocInBlock@CStdMalloc@@BECPEXLI@Z
 0001:24F4       ?AllocNewBlock@CStdMalloc@@BECLI@Z
 0001:3770       ?AssertValid@CArrayFValue@@RFCXXZ
 0001:4282       ?AssertValid@CMapKeyToValue@@RFCXXZ
 0003:015A       ?atfnProxy1632Vtbl@@3QEKE
 0001:15F8       ?CallbackHandler@@ZCHK@Z
 0001:1ABE       ?CallCanUnloadNow@@ZCKK@Z
 0001:1A80       ?CallGetClassObject@@ZCKPEUtagCALLGETCLASSOBJECTSTRUCT@@@Z
 0001:2B58       ?CallStub16@@ZCKPEUtagCallData@@@Z
 0001:1334       ?CheckIfMapEmpty@@ZAXXZ
 0001:3BBC       ?CompareAssocKey@CMapKeyToValue@@BFCHPEUCAssoc@1@PEXI@Z
 0001:4290       ?Create@CPlex@@TAPEU1@AEPEU1@KII@Z
 0001:2864       ?DidAlloc@CStdMalloc@@VEAHPEX@Z
 0001:27AE       ?Free@CStdMalloc@@VEAXPEX@Z
 0001:2F36       ?FreeAllLibraries@CDlls@@RECXXZ
 0001:28E4       ?FreeAllMem@CStdMalloc@@BECXXZ
 0001:3ADE       ?FreeAssoc@CMapKeyToValue@@BECXPEUCAssoc@1@@Z
 0001:3CEA       ?FreeAssocKey@CMapKeyToValue@@BFCXPEUCAssoc@1@@Z
 0001:42F4       ?FreeDataChain@CPlex@@RECXK@Z
 0001:3444       ?FreeExtra@CArrayFValue@@RECXXZ
 0001:2FA2       ?FreeUnusedLibraries@CDlls@@RECXXZ
 0002:0000       ?gdata16@@3UtagDATA16@@E
 0001:3B1E       ?GetAssocAt@CMapKeyToValue@@BFCPEUCAssoc@1@PEXIAEI@Z
 0001:3C94       ?GetAssocKeyPtr@CMapKeyToValue@@BFCXPEUCAssoc@1@PEPEXPEI@Z
 0001:3D46       ?GetAssocValue@CMapKeyToValue@@BFCXPEUCAssoc@1@PEX@Z
 0001:3D1E       ?GetAssocValuePtr@CMapKeyToValue@@BFCXPEUCAssoc@1@PEPEX@Z
 0001:4114       ?GetHKey@CMapKeyToValue@@RFCKPEXI@Z
 0001:2CE6       ?GetLibrary@CDlls@@RECIPEDH@Z
 0001:415C       ?GetNextAssoc@CMapKeyToValue@@RFCXPEPEXPEXPEI1@Z
 0001:3280       ?GetSize@CArrayFValue@@RFCHXZ
 0001:27F8       ?GetSize@CStdMalloc@@VEAKPEX@Z
 0001:413C       ?GetStartPosition@CMapKeyToValue@@RFCPEXXZ
 0001:28AA       ?HeapMinimize@CStdMalloc@@VEAXXZ
 0001:36A2       ?IndexOf@CArrayFValue@@RECHPEXII@Z
 0001:387E       ?InitHashTable@CMapKeyToValue@@BECHXZ
 0001:3568       ?InsertAt@CArrayFValue@@RECHHPEXH@Z
 0001:1318       ?IsValidEtask@@ZAHIAEUEtask@@@Z
 0001:19FC       ?LoadProcDll@@ZCKPEUtagLOADPROCDLLSTRUCT@@@Z
 0001:3DE2       ?Lookup@CMapKeyToValue@@RFCHPEXI0@Z
 0001:3E6E       ?LookupAdd@CMapKeyToValue@@RFCHPEXI0@Z
 0001:3E1C       ?LookupHKey@CMapKeyToValue@@RFCHKPEX@Z
 0003:049C       ?lpIUnknownObj32@@3PEXE
 0001:25B8       ?MapPtrToBlock@CStdMalloc@@BECLPEX@Z
 0001:28B6       ?MoveSelf@CStdMalloc@@BECPEV1@PEX@Z
 0001:39B2       ?NewAssoc@CMapKeyToValue@@BECPEUCAssoc@1@IPEXI0@Z
 0001:216C       ?Proxy1632AddRef@@ZAKPEVCProxy1632@@@Z
 0001:2282       ?Proxy1632Method10@@ZAKPEVCProxy1632@@@Z
 0001:229C       ?Proxy1632Method11@@ZAKPEVCProxy1632@@@Z
 0001:22B6       ?Proxy1632Method12@@ZAKPEVCProxy1632@@@Z
 0001:22D0       ?Proxy1632Method13@@ZAKPEVCProxy1632@@@Z
 0001:22EA       ?Proxy1632Method14@@ZAKPEVCProxy1632@@@Z
 0001:2304       ?Proxy1632Method15@@ZAKPEVCProxy1632@@@Z
 0001:231E       ?Proxy1632Method16@@ZAKPEVCProxy1632@@@Z
 0001:2338       ?Proxy1632Method17@@ZAKPEVCProxy1632@@@Z
 0001:2352       ?Proxy1632Method18@@ZAKPEVCProxy1632@@@Z
 0001:236C       ?Proxy1632Method19@@ZAKPEVCProxy1632@@@Z
 0001:2386       ?Proxy1632Method20@@ZAKPEVCProxy1632@@@Z
 0001:23A0       ?Proxy1632Method21@@ZAKPEVCProxy1632@@@Z
 0001:23BA       ?Proxy1632Method22@@ZAKPEVCProxy1632@@@Z
 0001:23D4       ?Proxy1632Method23@@ZAKPEVCProxy1632@@@Z
 0001:23EE       ?Proxy1632Method24@@ZAKPEVCProxy1632@@@Z
 0001:2408       ?Proxy1632Method25@@ZAKPEVCProxy1632@@@Z
 0001:2422       ?Proxy1632Method26@@ZAKPEVCProxy1632@@@Z
 0001:243C       ?Proxy1632Method27@@ZAKPEVCProxy1632@@@Z
 0001:2456       ?Proxy1632Method28@@ZAKPEVCProxy1632@@@Z
 0001:2470       ?Proxy1632Method29@@ZAKPEVCProxy1632@@@Z
 0001:248A       ?Proxy1632Method30@@ZAKPEVCProxy1632@@@Z
 0001:24A4       ?Proxy1632Method31@@ZAKPEVCProxy1632@@@Z
 0001:21CC       ?Proxy1632Method3@@ZAKPEVCProxy1632@@@Z
 0001:21E6       ?Proxy1632Method4@@ZAKPEVCProxy1632@@@Z
 0001:2200       ?Proxy1632Method5@@ZAKPEVCProxy1632@@@Z
 0001:221A       ?Proxy1632Method6@@ZAKPEVCProxy1632@@@Z
 0001:2234       ?Proxy1632Method7@@ZAKPEVCProxy1632@@@Z
 0001:224E       ?Proxy1632Method8@@ZAKPEVCProxy1632@@@Z
 0001:2268       ?Proxy1632Method9@@ZAKPEVCProxy1632@@@Z
 0001:20FE       ?Proxy1632QueryInterface@@ZAKPEVCProxy1632@@AFUGUID@@PEPEX@Z
 0001:219C       ?Proxy1632Release@@ZAKPEVCProxy1632@@@Z
 0001:1ADC       ?QueryInterface16@@ZCKPEUIUnknown@@AFUGUID@@PEPEX@Z
 0001:4F50       ?QueryInterface@CStdMalloc@@VEAPEXAFUGUID@@PEPEX@Z
 0001:268E       ?Realloc@CStdMalloc@@VEAPEXPEXK@Z
 0001:1C24       ?Release16@@ZCKPEUIUnknown@@@Z
 0001:501C       ?Release@CStdMalloc@@VEAKXZ
 0001:1450       ?ReleaseEtask@@ZAXIAEUEtask@@@Z
 0001:2EA8       ?ReleaseLibrary@CDlls@@RECXI@Z
 0001:1C54       ?ReleaseStgMedium16@@ZCKPEUtagSTGMEDIUM@@@Z
 0001:38F0       ?RemoveAll@CMapKeyToValue@@RECXXZ
 0001:364A       ?RemoveAt@CArrayFValue@@RECXHH@Z
 0001:406C       ?RemoveHKey@CMapKeyToValue@@RECHK@Z
 0001:3FAE       ?RemoveKey@CMapKeyToValue@@RECHPEXI@Z
 0001:3C10       ?SetAssocKey@CMapKeyToValue@@BFCHPEUCAssoc@1@PEXI@Z
 0001:3D84       ?SetAssocValue@CMapKeyToValue@@BFCXPEUCAssoc@1@PEX@Z
 0001:34F6       ?SetAt@CArrayFValue@@RECXHPEX@Z
 0001:3EB6       ?SetAt@CMapKeyToValue@@RECHPEXI0@Z
 0001:352A       ?SetAtGrow@CArrayFValue@@RECHHPEX@Z
 0001:3F72       ?SetAtHKey@CMapKeyToValue@@RECHKPEX@Z
 0001:1E78       ?SetOwnerPublic16@@ZCKK@Z
 0001:3296       ?SetSize@CArrayFValue@@RECHHH@Z
 0001:04C4       ?SetupSharedAllocator@@ZAHAEUEtask@@@Z
 0001:1C70       ?Sm16RhAddRef@@ZAKPEVCSm16ReleaseHandler@@@Z
 0001:1C92       ?Sm16RhQI@@ZAPEXPEVCSm16ReleaseHandler@@AFUGUID@@PEPEX@Z
 0001:1CE4       ?Sm16RhRelease@@ZAKPEVCSm16ReleaseHandler@@@Z
 0003:014E       ?Sm16RhVtbl@@3QEKE
 0001:1DDA       ?StgMediumStreamHandler16@@ZCKPEUIStream@@0@Z
 0001:040A       ?TaskAlloc@@ZCPEXK@Z
 0001:0476       ?TaskFree@@ZCXPEX@Z
 0001:1E4C       ?TouchPointer16@@ZCKPEE@Z
 0001:1A64       ?UnloadProcDll@@ZCKK@Z
 0003:045A       ?v_etaskCache@@3UEtask@@A
 0003:004E       ?v_hTaskCache@@3IE
 0003:043A       ?v_mapToEtask@@3VCMapHandleEtask@@A
 0003:0010       ?v_pidHighWord@@3IE
 0003:0016       ?v_pMallocPreShared@@3PEUIMalloc@@E
 0003:0012       ?v_pMallocShared@@3PEUIMalloc@@E
 0001:1E94       ?WinExec16@@ZCKPEUtagWINEXEC16STRUCT@@@Z
 0001:34D6       ?_GetAt@CArrayFValue@@RFCPEXH@Z
 0001:1F1C       ADDAPPCOMPATFLAG
 0001:162A       CALL32INITIALIZE
 0001:1814       CALL32UNINITIALIZE
 0001:18BC       CALLOBJECTINWOW
 0001:1954       CALLOBJECTINWOWCHECKINIT
 0001:19BC       CALLOBJECTINWOWCHECKTHKMGR
 0000:0000  Imp  CALLPROC32W          (KERNEL.CALLPROC32W)
 0001:188E       CALLTHKMGRINITIALIZE
 0001:1860       CALLTHKMGRUNINITIALIZE
 0001:1264       CLSIDFROMOLE1CLASS
 0001:023C       CLSIDFROMPROGID
 0001:0000       CLSIDFROMSTRING
 0001:0AB0       COBUILDVERSION
 0001:0262       COCREATEGUID
 0001:01CA       COCREATEINSTANCE
 0001:2946       COCREATESTANDARDMALLOC
 0001:0132       CODISCONNECTOBJECT
 0001:02AE       CODOSDATETIMETOFILETIME
 0001:02D4       COFILETIMENOW
 0001:0288       COFILETIMETODOSDATETIME
 0001:3186       COFREEALLLIBRARIES
 0001:315A       COFREELIBRARY
 0001:31BC       COFREEUNUSEDLIBRARIES
 0001:122E       COGETCLASSEXT
 0001:004E       COGETCLASSOBJECT
 0001:0A86       COGETCURRENTPROCESS
 0001:081E       COGETMALLOC
 0001:017E       COGETSTANDARDMARSHAL
 0001:093C       COGETSTATE
 0001:0320       COGETTREATASCLASS
 0001:12BE       COHANDLEINCOMINGCALL
 0001:056E       COINITIALIZE
 0001:01A4       COISHANDLERCONNECTED
 0001:01F0       COISOLE1CLASS
 0001:3128       COLOADLIBRARY
 0001:0158       COLOCKOBJECTEXTERNAL
 0001:0AC2       COMARSHALHRESULT
 0001:00C0       COMARSHALINTERFACE
 0001:2A74       COMEMALLOC
 0001:29F2       COMEMCTXOF
 0001:2AEC       COMEMFREE
 0001:1EB8       CONVERTHR1632
 0001:1EEA       CONVERTHR3216
 0001:1276       COOPENCLASSKEY
 0001:0074       COREGISTERCLASSOBJECT
 0001:02FA       COREGISTERMESSAGEFILTER
 0001:010C       CORELEASEMARSHALDATA
 0001:009A       COREVOKECLASSOBJECT
 0001:12AC       CORUNMODALLOOP
 0001:121C       COSETACKSTATE
 0001:09D6       COSETSTATE
 0001:0346       COTREATASCLASS
 0001:0796       COUNINITIALIZE
 0001:0B44       COUNMARSHALHRESULT
 0001:00E6       COUNMARSHALINTERFACE
 0000:0000  Imp  DELETEMETAFILE       (GDI.127)
 0000:0000  Imp  DOS3CALL             (KERNEL.102)
 0000:0000  Imp  FATALAPPEXIT         (KERNEL.137)
 0000:0000  Imp  FATALEXIT            (KERNEL.1)
 0001:119E       FNASSERT
 0000:0000  Imp  FREELIBRARY          (KERNEL.96)
 0000:0000  Imp  FREELIBRARY32W       (KERNEL.FREELIBRARY32W)
 0000:0000  Imp  GETCURRENTTASK       (KERNEL.36)
 0000:0000  Imp  GETDOSENVIRONMENT    (KERNEL.131)
 0000:0000  Imp  GETMODULEFILENAME    (KERNEL.49)
 0000:0000  Imp  GETPROCADDRESS       (KERNEL.50)
 0000:0000  Imp  GETPROCADDRESS32W    (KERNEL.GETPROCADDRESS32W)
 0000:0000  Imp  GETPROFILEINT        (KERNEL.57)
 0001:1148       GETSCODE
 0000:0000  Imp  GETVDMPOINTER32W     (KERNEL.GETVDMPOINTER32W)
 0000:0000  Imp  GETVERSION           (KERNEL.3)
 0000:0000  Imp  GLOBALALLOC          (KERNEL.15)
 0000:0000  Imp  GLOBALFREE           (KERNEL.17)
 0000:0000  Imp  GLOBALHANDLE         (KERNEL.21)
 0000:0000  Imp  GLOBALLOCK           (KERNEL.18)
 0000:0000  Imp  GLOBALREALLOC        (KERNEL.16)
 0000:0000  Imp  GLOBALSIZE           (KERNEL.20)
 0000:0000  Imp  GLOBALUNLOCK         (KERNEL.19)
 0001:0D3C       GUIDFROMSTRING
 0001:1050       IIDFROMSTRING
 0000:0000  Imp  INITAPP              (USER.5)
 0000:0000  Imp  INITTASK             (KERNEL.91)
 0000:0000  Imp  ISBADCODEPTR         (KERNEL.336)
 0000:0000  Imp  ISBADREADPTR         (KERNEL.334)
 0000:0000  Imp  ISBADWRITEPTR        (KERNEL.335)
 0001:0BE8       ISEQUALGUID
 0001:2C90       ISVALIDIID
 0001:2C22       ISVALIDINTERFACE
 0001:2BDA       ISVALIDPTRIN
 0001:2BFE       ISVALIDPTROUT
 0000:0000  Imp  KERNEL_SETOWNER      (KERNEL.403)
 0001:0388       LIBMAIN
 0000:0000  Imp  LOADLIBRARY          (KERNEL.95)
 0000:0000  Imp  LOADLIBRARYEX32W     (KERNEL.LOADLIBRARYEX32W)
 0000:0000  Imp  LOCALALLOC           (KERNEL.5)
 0000:0000  Imp  LOCALFREE            (KERNEL.7)
 0000:0000  Imp  LOCALINIT            (KERNEL.4)
 0000:0000  Imp  LOCALREALLOC         (KERNEL.6)
 0000:0000  Imp  LOCALSIZE            (KERNEL.10)
 0000:0000  Imp  LOCKSEGMENT          (KERNEL.23)
 0001:1344       LOOKUPETASK
 0001:1240       LRPCCALL
 0001:11B0       LRPCDISPATCH
 0001:11F8       LRPCFREEMONITORDATA
 0001:1288       LRPCGETTHREADWINDOW
 0001:1252       LRPCREGISTERMONITOR
 0001:129A       LRPCREVOKEMONITOR
 0001:383A       MKVDEFAULTHASHKEY
 0001:12E2       OLE1CLASSFROMCLSID2
 0001:0216       PROGIDFROMCLSID
 0001:1178       PROPAGATERESULT
 0000:0000  Imp  RELEASESTGMEDIUM     (OLE2.32)
 0001:11E6       REMALLOCOID
 0001:11C2       REMCONNECTTOOBJECT
 0001:11D4       REMCREATEREMOTEHANDLER
 0001:1306       REMFREEOID
 0001:12D0       REMGETINFOFORCID
 0001:12F4       REMLOOKUPSHUNK
 0001:157A       REMOVEETASK
 0001:1160       RESULTFROMSCODE
 0003:0004       rsrvptrs
 0000:0000  Imp  SETERRORMODE         (KERNEL.107)
 0001:13FE       SETETASK
 0001:1908       SSCALLOBJECTINWOW
 0000:0000  Imp  SSINIT               (KERNEL.700)
 0000:0000  Imp  SSONBIGSTACK         (KERNEL.701)
 0001:0EEC       STRINGFROMCLSID
 0001:10DE       STRINGFROMGUID2
 0001:0FA2       STRINGFROMIID
 0001:120A       TIMERCALLBACKPROC
 0000:0000  Imp  UNLOCKSEGMENT        (KERNEL.24)
 0000:0000  Imp  WAITEVENT            (KERNEL.30)
 0001:039E       WEP
 0000:0000  Imp  WINEXEC              (KERNEL.166)
 0003:021A       _aseghi
 0003:0218       _aseglo
 0001:4BBE       _atexit
 0001:1FAE       _CLSID_StdMarshal
 0003:043A       _edata
 0003:0550       _end
 0003:023C       _errno
 0001:4727       _exit
 0001:1F7E       _GUID_NULL
 0001:203E       _IID_IBindCtx
 0001:1F5E       _IID_IClassFactory
 0001:1FEE       _IID_IDfReserved1
 0001:1FDE       _IID_IDfReserved2
 0001:1FCE       _IID_IDfReserved3
 0001:204E       _IID_IEnumSTATSTG
 0001:1F8E       _IID_IExternalConnection
 0001:200E       _IID_IInternalMoniker
 0001:207E       _IID_ILockBytes
 0001:1F4E       _IID_IMalloc
 0001:20EE       _IID_IMarshal
 0001:1FBE       _IID_IMessageFilter
 0001:202E       _IID_IMoniker
 0000:0000  Imp  _IID_IOleContainer   (OLE2.147)
 0000:0000  Imp  _IID_IOleItemContainer (OLE2.148)
 0000:0000  Imp  _IID_IPersist        (OLE2.132)
 0000:0000  Imp  _IID_IPersistFile    (OLE2.131)
 0000:0000  Imp  _IID_IPersistStorage (OLE2.130)
 0000:0000  Imp  _IID_IPersistStream  (OLE2.129)
 0001:209E       _IID_IProxyManager
 0001:208E       _IID_IPSFactory
 0001:1FFE       _IID_IRootStorage
 0001:20DE       _IID_IRpcChannel
 0001:20AE       _IID_IRpcProxy
 0001:20CE       _IID_IRpcStub
 0001:201E       _IID_IRunningObjectTable
 0001:1F9E       _IID_IStdMarshalInfo
 0001:206E       _IID_IStorage
 0001:205E       _IID_IStream
 0001:20BE       _IID_IStubManager
 0001:1F6E       _IID_IUnknown
 0000:0000  Imp  _SSCALL              (KERNEL.702)
 0003:020C       _STKHQQ
 0000:0000  Imp  _wsprintf            (USER.420)
 0003:0220       __acfinfo
 0000:9876  Abs  __acrtmsg
 0000:9876  Abs  __acrtused
 0000:D6D6  Abs  __aDBdoswp
 0003:028E       __adbgmsg
 0000:D6D6  Abs  __aDBused
 0001:4B9E       __aFahdiff
 0001:4440       __aFlshl
 0000:0000  Imp  __AHINCR             (KERNEL.114)
 0000:0000  Imp  __AHSHIFT            (KERNEL.113)
 0003:022E       __aintdiv
 0003:02AC       __amblksiz
 0001:4A94       __amsg_exit
 0001:435A       __astart
 0001:4744       __cexit
 0003:028B       __child
 0001:4644       __cinit
 0001:4A8A       __cintDIV
 0003:0216       __cmdShow
 0003:024B       __cpumode
 0001:47C5       __ctermsub
 0001:4755       __c_exit
 0003:024C       __doserrno
 0003:043A       __edata
 0003:0550       __end
 0003:0282       __environ
 0001:4735       __exit
 0003:028D       __exitflag
 0003:0232       __fac
 0001:4AD6       __ffree
 0001:4802       __FF_MSGBANNER
 0003:029E       __fheap
 0001:4E27       __findlast
 0001:4AF7       __fmalloc
 0001:444C       __fmemcmp
 0001:44A8       __fmemcpy
 0001:454E       __fmemmove
 0001:4506       __fmemset
 0003:02B4       __fpinit
 0000:9876  Abs  __fptaskdata
 0001:4BFC       __fptrap
 0001:443A       __fpurecall
 0001:4CA4       __GetDGROUP
 0001:4D30       __growseg
 0003:0210       __hInstance
 0003:020E       __hPrevInstance
 0001:4DC1       __incseg
 0001:4EDE       __initseg
 0001:4F12       __linkseg
 0003:0212       __lpszCmdLine
 0001:4C76       __myalloc
 0001:4E48       __newseg
 0003:024E       __nfile
 0001:4C02       __NMSG_TEXT
 0001:4C39       __NMSG_WRITE
 0001:4411       __nomain
 0001:443A       __npurecall
 0001:4BC6       __onexit
 0003:024C       __oserr
 0003:0254       __osfile
 0003:0247       __osmajor
 0003:0246       __osminor
 0003:024A       __osmode
 0003:0246       __osver
 0003:0248       __osversion
 0003:0286       __pgmptr
 0003:0296       __pnhFarHeap
 0003:0242       __psp
 0003:0240       __pspadr
 0001:443A       __purecall
 0001:4BF5       __QWINClose
 0001:4BF5       __QWINExit
 0001:4BF5       __QWINGetBuffSize
 0001:4BF5       __QWINGetFocus
 0001:4BF5       __QWINGetSize
 0001:4BF5       __QWINInit
 0001:4BF5       __QWINIsQWINin
 0001:4BF5       __QWINMenuClick
 0001:4BF5       __QWINOpen
 0001:4BF5       __QWINRead
 0001:4BF5       __QWINSetAboutString
 0001:4BF5       __QWINSetBuffSize
 0001:4BF5       __QWINSetFocus
 0001:4BF5       __QWINSetSize
 0001:4BF5       __QWINTerm
 0003:029C       __qwinused
 0001:4BF5       __QWINWrite
 0001:4BF5       __QWINYield
 0001:4CB4       __searchseg
 0001:4826       __setargv
 0001:49D0       __setenvp
 0000:0001  Abs  __sizec
 0000:0001  Abs  __sized
 0001:4618       __stubmain
 0003:023E       __umaskval
 0001:4BF5       __wabout
 0001:4BF0       __wcexit
 0001:4BF0       __wcinit
 0001:4BF5       __wclose
 0003:0250       __wfile
 0001:4350       __wflags
 0001:4BF5       __wgetfocus
 0001:4BF5       __wgetscreenbuf
 0001:4BF5       __wgetsize
 0000:0000  Imp  __WINFLAGS           (KERNEL.178)
 0003:0245       __winmajor
 0003:0244       __winminor
 0003:0244       __winver
 0000:0000  Abs  __wiobused
 0001:4BF5       __wmenuclick
 0003:0252       __wnfile
 0001:4BF5       __wopen
 0001:4BF5       __wread
 0001:4BF5       __wsetfocus
 0001:4BF5       __wsetscreenbuf
 0001:4BF5       __wsetsize
 0003:0268       __wsfile
 0001:4BF5       __wterm
 0001:4BF5       __wwrite
 0003:021E       ___aDBrterr
 0003:021C       ___aDBswpflg
 0003:027C       ___argc
 0003:027E       ___argv
 0001:4ECA       ___ExportedStub

  Address         Publics by Value

 0000:0000  Abs  __wiobused
 0000:0000  Imp  LOCKSEGMENT          (KERNEL.23)
 0000:0000  Imp  GETPROCADDRESS       (KERNEL.50)
 0000:0000  Imp  _IID_IOleContainer   (OLE2.147)
 0000:0000  Imp  KERNEL_SETOWNER      (KERNEL.403)
 0000:0000  Imp  _wsprintf            (USER.420)
 0000:0000  Imp  GETDOSENVIRONMENT    (KERNEL.131)
 0000:0000  Imp  WAITEVENT            (KERNEL.30)
 0000:0000  Imp  FATALAPPEXIT         (KERNEL.137)
 0000:0000  Imp  RELEASESTGMEDIUM     (OLE2.32)
 0000:0000  Imp  CALLPROC32W          (KERNEL.CALLPROC32W)
 0000:0000  Imp  GLOBALFREE           (KERNEL.17)
 0000:0000  Imp  GLOBALSIZE           (KERNEL.20)
 0000:0000  Imp  _SSCALL              (KERNEL.702)
 0000:0000  Imp  SETERRORMODE         (KERNEL.107)
 0000:0000  Imp  GETPROFILEINT        (KERNEL.57)
 0000:0000  Imp  __AHINCR             (KERNEL.114)
 0000:0000  Imp  SSINIT               (KERNEL.700)
 0000:0000  Imp  GETMODULEFILENAME    (KERNEL.49)
 0000:0000  Imp  LOCALINIT            (KERNEL.4)
 0000:0000  Imp  ISBADCODEPTR         (KERNEL.336)
 0000:0000  Imp  LOADLIBRARY          (KERNEL.95)
 0000:0000  Imp  FATALEXIT            (KERNEL.1)
 0000:0000  Imp  GETCURRENTTASK       (KERNEL.36)
 0000:0000  Imp  ISBADREADPTR         (KERNEL.334)
 0000:0000  Imp  LOADLIBRARYEX32W     (KERNEL.LOADLIBRARYEX32W)
 0000:0000  Imp  DELETEMETAFILE       (GDI.127)
 0000:0000  Imp  GLOBALALLOC          (KERNEL.15)
 0000:0000  Imp  DOS3CALL             (KERNEL.102)
 0000:0000  Imp  ISBADWRITEPTR        (KERNEL.335)
 0000:0000  Imp  _IID_IOleItemContainer (OLE2.148)
 0000:0000  Imp  LOCALALLOC           (KERNEL.5)
 0000:0000  Imp  SSONBIGSTACK         (KERNEL.701)
 0000:0000  Imp  GLOBALLOCK           (KERNEL.18)
 0000:0000  Imp  LOCALREALLOC         (KERNEL.6)
 0000:0000  Imp  UNLOCKSEGMENT        (KERNEL.24)
 0000:0000  Imp  GETVERSION           (KERNEL.3)
 0000:0000  Imp  __AHSHIFT            (KERNEL.113)
 0000:0000  Imp  __WINFLAGS           (KERNEL.178)
 0000:0000  Imp  WINEXEC              (KERNEL.166)
 0000:0000  Imp  _IID_IPersistStream  (OLE2.129)
 0000:0000  Imp  LOCALFREE            (KERNEL.7)
 0000:0000  Imp  _IID_IPersist        (OLE2.132)
 0000:0000  Imp  GETVDMPOINTER32W     (KERNEL.GETVDMPOINTER32W)
 0000:0000  Imp  _IID_IPersistFile    (OLE2.131)
 0000:0000  Imp  GETPROCADDRESS32W    (KERNEL.GETPROCADDRESS32W)
 0000:0000  Imp  FREELIBRARY32W       (KERNEL.FREELIBRARY32W)
 0000:0000  Imp  FREELIBRARY          (KERNEL.96)
 0000:0000  Imp  GLOBALUNLOCK         (KERNEL.19)
 0000:0000  Imp  INITTASK             (KERNEL.91)
 0000:0000  Imp  _IID_IPersistStorage (OLE2.130)
 0000:0000  Imp  LOCALSIZE            (KERNEL.10)
 0000:0000  Imp  GLOBALREALLOC        (KERNEL.16)
 0000:0000  Imp  GLOBALHANDLE         (KERNEL.21)
 0000:0000  Imp  INITAPP              (USER.5)
 0000:0001  Abs  __sized
 0000:0001  Abs  __sizec
 0000:9876  Abs  __fptaskdata
 0000:9876  Abs  __acrtused
 0000:9876  Abs  __acrtmsg
 0000:D6D6  Abs  __aDBused
 0000:D6D6  Abs  __aDBdoswp
 0001:0000       CLSIDFROMSTRING
 0001:004E       COGETCLASSOBJECT
 0001:0074       COREGISTERCLASSOBJECT
 0001:009A       COREVOKECLASSOBJECT
 0001:00C0       COMARSHALINTERFACE
 0001:00E6       COUNMARSHALINTERFACE
 0001:010C       CORELEASEMARSHALDATA
 0001:0132       CODISCONNECTOBJECT
 0001:0158       COLOCKOBJECTEXTERNAL
 0001:017E       COGETSTANDARDMARSHAL
 0001:01A4       COISHANDLERCONNECTED
 0001:01CA       COCREATEINSTANCE
 0001:01F0       COISOLE1CLASS
 0001:0216       PROGIDFROMCLSID
 0001:023C       CLSIDFROMPROGID
 0001:0262       COCREATEGUID
 0001:0288       COFILETIMETODOSDATETIME
 0001:02AE       CODOSDATETIMETOFILETIME
 0001:02D4       COFILETIMENOW
 0001:02FA       COREGISTERMESSAGEFILTER
 0001:0320       COGETTREATASCLASS
 0001:0346       COTREATASCLASS
 0001:0388       LIBMAIN
 0001:039E       WEP
 0001:040A       ?TaskAlloc@@ZCPEXK@Z
 0001:0476       ?TaskFree@@ZCXPEX@Z
 0001:04C4       ?SetupSharedAllocator@@ZAHAEUEtask@@@Z
 0001:056E       COINITIALIZE
 0001:0796       COUNINITIALIZE
 0001:081E       COGETMALLOC
 0001:093C       COGETSTATE
 0001:09D6       COSETSTATE
 0001:0A86       COGETCURRENTPROCESS
 0001:0AB0       COBUILDVERSION
 0001:0AC2       COMARSHALHRESULT
 0001:0B44       COUNMARSHALHRESULT
 0001:0BE8       ISEQUALGUID
 0001:0D3C       GUIDFROMSTRING
 0001:0EEC       STRINGFROMCLSID
 0001:0FA2       STRINGFROMIID
 0001:1050       IIDFROMSTRING
 0001:10DE       STRINGFROMGUID2
 0001:1148       GETSCODE
 0001:1160       RESULTFROMSCODE
 0001:1178       PROPAGATERESULT
 0001:119E       FNASSERT
 0001:11B0       LRPCDISPATCH
 0001:11C2       REMCONNECTTOOBJECT
 0001:11D4       REMCREATEREMOTEHANDLER
 0001:11E6       REMALLOCOID
 0001:11F8       LRPCFREEMONITORDATA
 0001:120A       TIMERCALLBACKPROC
 0001:121C       COSETACKSTATE
 0001:122E       COGETCLASSEXT
 0001:1240       LRPCCALL
 0001:1252       LRPCREGISTERMONITOR
 0001:1264       CLSIDFROMOLE1CLASS
 0001:1276       COOPENCLASSKEY
 0001:1288       LRPCGETTHREADWINDOW
 0001:129A       LRPCREVOKEMONITOR
 0001:12AC       CORUNMODALLOOP
 0001:12BE       COHANDLEINCOMINGCALL
 0001:12D0       REMGETINFOFORCID
 0001:12E2       OLE1CLASSFROMCLSID2
 0001:12F4       REMLOOKUPSHUNK
 0001:1306       REMFREEOID
 0001:1318       ?IsValidEtask@@ZAHIAEUEtask@@@Z
 0001:1334       ?CheckIfMapEmpty@@ZAXXZ
 0001:1344       LOOKUPETASK
 0001:13FE       SETETASK
 0001:1450       ?ReleaseEtask@@ZAXIAEUEtask@@@Z
 0001:157A       REMOVEETASK
 0001:15F8       ?CallbackHandler@@ZCHK@Z
 0001:162A       CALL32INITIALIZE
 0001:1814       CALL32UNINITIALIZE
 0001:1860       CALLTHKMGRUNINITIALIZE
 0001:188E       CALLTHKMGRINITIALIZE
 0001:18BC       CALLOBJECTINWOW
 0001:1908       SSCALLOBJECTINWOW
 0001:1954       CALLOBJECTINWOWCHECKINIT
 0001:19BC       CALLOBJECTINWOWCHECKTHKMGR
 0001:19FC       ?LoadProcDll@@ZCKPEUtagLOADPROCDLLSTRUCT@@@Z
 0001:1A64       ?UnloadProcDll@@ZCKK@Z
 0001:1A80       ?CallGetClassObject@@ZCKPEUtagCALLGETCLASSOBJECTSTRUCT@@@Z
 0001:1ABE       ?CallCanUnloadNow@@ZCKK@Z
 0001:1ADC       ?QueryInterface16@@ZCKPEUIUnknown@@AFUGUID@@PEPEX@Z
 0001:1BF4       ?AddRef16@@ZCKPEUIUnknown@@@Z
 0001:1C24       ?Release16@@ZCKPEUIUnknown@@@Z
 0001:1C54       ?ReleaseStgMedium16@@ZCKPEUtagSTGMEDIUM@@@Z
 0001:1C70       ?Sm16RhAddRef@@ZAKPEVCSm16ReleaseHandler@@@Z
 0001:1C92       ?Sm16RhQI@@ZAPEXPEVCSm16ReleaseHandler@@AFUGUID@@PEPEX@Z
 0001:1CE4       ?Sm16RhRelease@@ZAKPEVCSm16ReleaseHandler@@@Z
 0001:1DDA       ?StgMediumStreamHandler16@@ZCKPEUIStream@@0@Z
 0001:1E4C       ?TouchPointer16@@ZCKPEE@Z
 0001:1E78       ?SetOwnerPublic16@@ZCKK@Z
 0001:1E94       ?WinExec16@@ZCKPEUtagWINEXEC16STRUCT@@@Z
 0001:1EB8       CONVERTHR1632
 0001:1EEA       CONVERTHR3216
 0001:1F1C       ADDAPPCOMPATFLAG
 0001:1F4E       _IID_IMalloc
 0001:1F5E       _IID_IClassFactory
 0001:1F6E       _IID_IUnknown
 0001:1F7E       _GUID_NULL
 0001:1F8E       _IID_IExternalConnection
 0001:1F9E       _IID_IStdMarshalInfo
 0001:1FAE       _CLSID_StdMarshal
 0001:1FBE       _IID_IMessageFilter
 0001:1FCE       _IID_IDfReserved3
 0001:1FDE       _IID_IDfReserved2
 0001:1FEE       _IID_IDfReserved1
 0001:1FFE       _IID_IRootStorage
 0001:200E       _IID_IInternalMoniker
 0001:201E       _IID_IRunningObjectTable
 0001:202E       _IID_IMoniker
 0001:203E       _IID_IBindCtx
 0001:204E       _IID_IEnumSTATSTG
 0001:205E       _IID_IStream
 0001:206E       _IID_IStorage
 0001:207E       _IID_ILockBytes
 0001:208E       _IID_IPSFactory
 0001:209E       _IID_IProxyManager
 0001:20AE       _IID_IRpcProxy
 0001:20BE       _IID_IStubManager
 0001:20CE       _IID_IRpcStub
 0001:20DE       _IID_IRpcChannel
 0001:20EE       _IID_IMarshal
 0001:20FE       ?Proxy1632QueryInterface@@ZAKPEVCProxy1632@@AFUGUID@@PEPEX@Z
 0001:216C       ?Proxy1632AddRef@@ZAKPEVCProxy1632@@@Z
 0001:219C       ?Proxy1632Release@@ZAKPEVCProxy1632@@@Z
 0001:21CC       ?Proxy1632Method3@@ZAKPEVCProxy1632@@@Z
 0001:21E6       ?Proxy1632Method4@@ZAKPEVCProxy1632@@@Z
 0001:2200       ?Proxy1632Method5@@ZAKPEVCProxy1632@@@Z
 0001:221A       ?Proxy1632Method6@@ZAKPEVCProxy1632@@@Z
 0001:2234       ?Proxy1632Method7@@ZAKPEVCProxy1632@@@Z
 0001:224E       ?Proxy1632Method8@@ZAKPEVCProxy1632@@@Z
 0001:2268       ?Proxy1632Method9@@ZAKPEVCProxy1632@@@Z
 0001:2282       ?Proxy1632Method10@@ZAKPEVCProxy1632@@@Z
 0001:229C       ?Proxy1632Method11@@ZAKPEVCProxy1632@@@Z
 0001:22B6       ?Proxy1632Method12@@ZAKPEVCProxy1632@@@Z
 0001:22D0       ?Proxy1632Method13@@ZAKPEVCProxy1632@@@Z
 0001:22EA       ?Proxy1632Method14@@ZAKPEVCProxy1632@@@Z
 0001:2304       ?Proxy1632Method15@@ZAKPEVCProxy1632@@@Z
 0001:231E       ?Proxy1632Method16@@ZAKPEVCProxy1632@@@Z
 0001:2338       ?Proxy1632Method17@@ZAKPEVCProxy1632@@@Z
 0001:2352       ?Proxy1632Method18@@ZAKPEVCProxy1632@@@Z
 0001:236C       ?Proxy1632Method19@@ZAKPEVCProxy1632@@@Z
 0001:2386       ?Proxy1632Method20@@ZAKPEVCProxy1632@@@Z
 0001:23A0       ?Proxy1632Method21@@ZAKPEVCProxy1632@@@Z
 0001:23BA       ?Proxy1632Method22@@ZAKPEVCProxy1632@@@Z
 0001:23D4       ?Proxy1632Method23@@ZAKPEVCProxy1632@@@Z
 0001:23EE       ?Proxy1632Method24@@ZAKPEVCProxy1632@@@Z
 0001:2408       ?Proxy1632Method25@@ZAKPEVCProxy1632@@@Z
 0001:2422       ?Proxy1632Method26@@ZAKPEVCProxy1632@@@Z
 0001:243C       ?Proxy1632Method27@@ZAKPEVCProxy1632@@@Z
 0001:2456       ?Proxy1632Method28@@ZAKPEVCProxy1632@@@Z
 0001:2470       ?Proxy1632Method29@@ZAKPEVCProxy1632@@@Z
 0001:248A       ?Proxy1632Method30@@ZAKPEVCProxy1632@@@Z
 0001:24A4       ?Proxy1632Method31@@ZAKPEVCProxy1632@@@Z
 0001:24BE       ?AllocInBlock@CStdMalloc@@BECPEXLI@Z
 0001:24F4       ?AllocNewBlock@CStdMalloc@@BECLI@Z
 0001:25B8       ?MapPtrToBlock@CStdMalloc@@BECLPEX@Z
 0001:2610       ?Alloc@CStdMalloc@@VEAPEXK@Z
 0001:268E       ?Realloc@CStdMalloc@@VEAPEXPEXK@Z
 0001:27AE       ?Free@CStdMalloc@@VEAXPEX@Z
 0001:27F8       ?GetSize@CStdMalloc@@VEAKPEX@Z
 0001:2864       ?DidAlloc@CStdMalloc@@VEAHPEX@Z
 0001:28AA       ?HeapMinimize@CStdMalloc@@VEAXXZ
 0001:28B6       ?MoveSelf@CStdMalloc@@BECPEV1@PEX@Z
 0001:28E4       ?FreeAllMem@CStdMalloc@@BECXXZ
 0001:2946       COCREATESTANDARDMALLOC
 0001:29F2       COMEMCTXOF
 0001:2A74       COMEMALLOC
 0001:2AEC       COMEMFREE
 0001:2B58       ?CallStub16@@ZCKPEUtagCallData@@@Z
 0001:2BDA       ISVALIDPTRIN
 0001:2BFE       ISVALIDPTROUT
 0001:2C22       ISVALIDINTERFACE
 0001:2C90       ISVALIDIID
 0001:2CE6       ?GetLibrary@CDlls@@RECIPEDH@Z
 0001:2EA8       ?ReleaseLibrary@CDlls@@RECXI@Z
 0001:2F36       ?FreeAllLibraries@CDlls@@RECXXZ
 0001:2FA2       ?FreeUnusedLibraries@CDlls@@RECXXZ
 0001:3128       COLOADLIBRARY
 0001:315A       COFREELIBRARY
 0001:3186       COFREEALLLIBRARIES
 0001:31BC       COFREEUNUSEDLIBRARIES
 0001:31FC       ??0CArrayFValue@@REC@KI@Z
 0001:325A       ??1CArrayFValue@@REC@XZ
 0001:3280       ?GetSize@CArrayFValue@@RFCHXZ
 0001:3296       ?SetSize@CArrayFValue@@RECHHH@Z
 0001:3444       ?FreeExtra@CArrayFValue@@RECXXZ
 0001:34D6       ?_GetAt@CArrayFValue@@RFCPEXH@Z
 0001:34F6       ?SetAt@CArrayFValue@@RECXHPEX@Z
 0001:352A       ?SetAtGrow@CArrayFValue@@RECHHPEX@Z
 0001:3568       ?InsertAt@CArrayFValue@@RECHHPEXH@Z
 0001:364A       ?RemoveAt@CArrayFValue@@RECXHH@Z
 0001:36A2       ?IndexOf@CArrayFValue@@RECHPEXII@Z
 0001:3770       ?AssertValid@CArrayFValue@@RFCXXZ
 0001:377E       ??0CMapKeyToValue@@REC@KIIHP7CIPEXI@ZI@Z
 0001:3822       ??1CMapKeyToValue@@REC@XZ
 0001:383A       MKVDEFAULTHASHKEY
 0001:387E       ?InitHashTable@CMapKeyToValue@@BECHXZ
 0001:38F0       ?RemoveAll@CMapKeyToValue@@RECXXZ
 0001:39B2       ?NewAssoc@CMapKeyToValue@@BECPEUCAssoc@1@IPEXI0@Z
 0001:3ADE       ?FreeAssoc@CMapKeyToValue@@BECXPEUCAssoc@1@@Z
 0001:3B1E       ?GetAssocAt@CMapKeyToValue@@BFCPEUCAssoc@1@PEXIAEI@Z
 0001:3BBC       ?CompareAssocKey@CMapKeyToValue@@BFCHPEUCAssoc@1@PEXI@Z
 0001:3C10       ?SetAssocKey@CMapKeyToValue@@BFCHPEUCAssoc@1@PEXI@Z
 0001:3C94       ?GetAssocKeyPtr@CMapKeyToValue@@BFCXPEUCAssoc@1@PEPEXPEI@Z
 0001:3CEA       ?FreeAssocKey@CMapKeyToValue@@BFCXPEUCAssoc@1@@Z
 0001:3D1E       ?GetAssocValuePtr@CMapKeyToValue@@BFCXPEUCAssoc@1@PEPEX@Z
 0001:3D46       ?GetAssocValue@CMapKeyToValue@@BFCXPEUCAssoc@1@PEX@Z
 0001:3D84       ?SetAssocValue@CMapKeyToValue@@BFCXPEUCAssoc@1@PEX@Z
 0001:3DE2       ?Lookup@CMapKeyToValue@@RFCHPEXI0@Z
 0001:3E1C       ?LookupHKey@CMapKeyToValue@@RFCHKPEX@Z
 0001:3E6E       ?LookupAdd@CMapKeyToValue@@RFCHPEXI0@Z
 0001:3EB6       ?SetAt@CMapKeyToValue@@RECHPEXI0@Z
 0001:3F72       ?SetAtHKey@CMapKeyToValue@@RECHKPEX@Z
 0001:3FAE       ?RemoveKey@CMapKeyToValue@@RECHPEXI@Z
 0001:406C       ?RemoveHKey@CMapKeyToValue@@RECHK@Z
 0001:4114       ?GetHKey@CMapKeyToValue@@RFCKPEXI@Z
 0001:413C       ?GetStartPosition@CMapKeyToValue@@RFCPEXXZ
 0001:415C       ?GetNextAssoc@CMapKeyToValue@@RFCXPEPEXPEXPEI1@Z
 0001:4282       ?AssertValid@CMapKeyToValue@@RFCXXZ
 0001:4290       ?Create@CPlex@@TAPEU1@AEPEU1@KII@Z
 0001:42F4       ?FreeDataChain@CPlex@@RECXK@Z
 0001:4350       __wflags
 0001:435A       __astart
 0001:4411       __nomain
 0001:4418       ??3@ZAXPEX@Z
 0001:442A       ??2@ZAPEXI@Z
 0001:443A       __npurecall
 0001:443A       __fpurecall
 0001:443A       __purecall
 0001:4440       __aFlshl
 0001:444C       __fmemcmp
 0001:44A8       __fmemcpy
 0001:4506       __fmemset
 0001:454E       __fmemmove
 0001:4618       __stubmain
 0001:4644       __cinit
 0001:4727       _exit
 0001:4735       __exit
 0001:4744       __cexit
 0001:4755       __c_exit
 0001:47C5       __ctermsub
 0001:4802       __FF_MSGBANNER
 0001:4826       __setargv
 0001:49D0       __setenvp
 0001:4A8A       __cintDIV
 0001:4A94       __amsg_exit
 0001:4AD6       __ffree
 0001:4AF7       __fmalloc
 0001:4B9E       __aFahdiff
 0001:4BBE       _atexit
 0001:4BC6       __onexit
 0001:4BF0       __wcexit
 0001:4BF0       __wcinit
 0001:4BF5       __QWINRead
 0001:4BF5       __wgetfocus
 0001:4BF5       __wgetscreenbuf
 0001:4BF5       __wread
 0001:4BF5       __QWINWrite
 0001:4BF5       __QWINMenuClick
 0001:4BF5       __wmenuclick
 0001:4BF5       __QWINExit
 0001:4BF5       __QWINClose
 0001:4BF5       __wsetsize
 0001:4BF5       __wopen
 0001:4BF5       __wgetsize
 0001:4BF5       __wterm
 0001:4BF5       __wwrite
 0001:4BF5       __QWINGetSize
 0001:4BF5       __wsetscreenbuf
 0001:4BF5       __QWINSetSize
 0001:4BF5       __QWINInit
 0001:4BF5       __wsetfocus
 0001:4BF5       __wclose
 0001:4BF5       __QWINSetFocus
 0001:4BF5       __QWINGetFocus
 0001:4BF5       __QWINSetAboutString
 0001:4BF5       __QWINSetBuffSize
 0001:4BF5       __QWINYield
 0001:4BF5       __QWINIsQWINin
 0001:4BF5       __QWINTerm
 0001:4BF5       __QWINGetBuffSize
 0001:4BF5       __wabout
 0001:4BF5       __QWINOpen
 0001:4BFC       __fptrap
 0001:4C02       __NMSG_TEXT
 0001:4C39       __NMSG_WRITE
 0001:4C76       __myalloc
 0001:4CA4       __GetDGROUP
 0001:4CB4       __searchseg
 0001:4D30       __growseg
 0001:4DC1       __incseg
 0001:4E27       __findlast
 0001:4E48       __newseg
 0001:4ECA       ___ExportedStub
 0001:4EDE       __initseg
 0001:4F12       __linkseg
 0001:4F50       ?QueryInterface@CStdMalloc@@VEAPEXAFUGUID@@PEPEX@Z
 0001:4FFA       ?AddRef@CStdMalloc@@VEAKXZ
 0001:501C       ?Release@CStdMalloc@@VEAKXZ
 0001:5058       ??0IMalloc@@REC@XZ
 0001:5080       ??_7IUnknown@@6F@
 0001:508C       ??_7IMalloc@@6F@
 0001:50B0       ??_7CStdMalloc@@6F@
 0002:0000       ?gdata16@@3UtagDATA16@@E
 0003:0004       rsrvptrs
 0003:0010       ?v_pidHighWord@@3IE
 0003:0012       ?v_pMallocShared@@3PEUIMalloc@@E
 0003:0016       ?v_pMallocPreShared@@3PEUIMalloc@@E
 0003:004E       ?v_hTaskCache@@3IE
 0003:014E       ?Sm16RhVtbl@@3QEKE
 0003:015A       ?atfnProxy1632Vtbl@@3QEKE
 0003:020C       _STKHQQ
 0003:020E       __hPrevInstance
 0003:0210       __hInstance
 0003:0212       __lpszCmdLine
 0003:0216       __cmdShow
 0003:0218       _aseglo
 0003:021A       _aseghi
 0003:021C       ___aDBswpflg
 0003:021E       ___aDBrterr
 0003:0220       __acfinfo
 0003:022E       __aintdiv
 0003:0232       __fac
 0003:023C       _errno
 0003:023E       __umaskval
 0003:0240       __pspadr
 0003:0242       __psp
 0003:0244       __winminor
 0003:0244       __winver
 0003:0245       __winmajor
 0003:0246       __osminor
 0003:0246       __osver
 0003:0247       __osmajor
 0003:0248       __osversion
 0003:024A       __osmode
 0003:024B       __cpumode
 0003:024C       __doserrno
 0003:024C       __oserr
 0003:024E       __nfile
 0003:0250       __wfile
 0003:0252       __wnfile
 0003:0254       __osfile
 0003:0268       __wsfile
 0003:027C       ___argc
 0003:027E       ___argv
 0003:0282       __environ
 0003:0286       __pgmptr
 0003:028B       __child
 0003:028D       __exitflag
 0003:028E       __adbgmsg
 0003:0296       __pnhFarHeap
 0003:029C       __qwinused
 0003:029E       __fheap
 0003:02AC       __amblksiz
 0003:02B4       __fpinit
 0003:043A       _edata
 0003:043A       ?v_mapToEtask@@3VCMapHandleEtask@@A
 0003:043A       __edata
 0003:045A       ?v_etaskCache@@3UEtask@@A
 0003:049C       ?lpIUnknownObj32@@3PEXE
 0003:0550       _end
 0003:0550       __end

Program entry point at 0001:435a
